:100000002CC056C009C154C053C057C051C050C0C5
:100010004FC04EC04DC04CC0CFC04AC049C0000008
:1000200000000000000000000000000023456C9864
:10003000C9FF040714233764A0FFFFFFFFFFFFFF82
:10004000FFFFFFFFFF000000000000000000234052
:100050005F7AB4FFFFFFFFFFFF0011241FBECFE553
:10006000D2E0DEBFCDBF20E0A0E6B0E001C01D922F
:10007000A738B207E1F7E2E6F0E085E5808781E0A6
:1000800083831482128286831182ADE6B0E08EEF04
:1000900015968C9315978DEF17968C938BE081872F
:1000A00088E58287612C712C88248A9486D0E2C0EE
:1000B000A7CF1BBC19BC18BC0895189525B7277E7F
:1000C00025BF29B7226029BF21E022BF019728F070
:1000D00020E188952150E9F7F9CF089588EE93E063
:1000E000EDCF8CE287B986EC86B9369A3699FECF89
:1000F0008FEF809360000895369A3699FECF95B1C0
:100100008091600089270895811101C0D2CF81506C
:1001100090E0FC01E25EFF4FE491EBBDFC01EE5C80
:10012000FF4FE491E9BDFC01EA5BFF4F849188BD7C
:1001300008950F931F93CF93C82F8B01CC2359F0B1
:1001400085E0E2DFC801BADFB4DFC801B7DFC8016C
:10015000B5DFC150F3CFCF911F910F910895CF9389
:10016000DF93D82F64E170E08AE0E3DF84EF91E071
:10017000A5DF8D2F64E672D0CAE06C2F6FD0892F77
:1001800068EC70E0D6DFAADF8D2F6C2F67D0D92FF7
:1001900065D0892F68EC70E0CCDFA0DF68EC70E000
:1001A0008D2FC7DF9BDF64E170E08AE0C2DF84EF60
:1001B00091E0DF91CF9182CF18958FE384BBB99AFC
:1001C000B89ABC9A81E08ABD83BF9AB590629ABD05
:1001D0009AB590689ABD9FEF9DBD80BF80E68CBDAB
:1001E00097B328B3892F90E0809590958B7F822BD1
:1001F00088BBC298AA9A8BB780628BBF8AB785608A
:100200008ABF85B7806285BF78946BDF8CE291E00E
:1002100055DF72DFA4DFFACF1124882009F018958A
:10022000F89416B846DFB998B898BC9894E4B29997
:100230000FC0839485B7877E806185BF91BD85B7E8
:10024000846885BF8B7F85BF78948895F894EFCFBD
:100250008FE58DBF82E08EBF1FBEAFDF991B79E0B7
:1002600004C0991F961708F0961B881F7A95C9F746
:0802700080950895F894FFCF7A
:00000001FF
